:100000000AC0189518951895189523C2C6C018955A
:100010001895189518958FE181BD87E181BD8FED09
:100020008DBFC8EBE4EA4E2EDD275D2EEEE7F0E053
:10003000A0E6B0E088278D933197E9F766248FEF2B
:1000400087BB8CE381BB83E482BB83E083BF89B73A
:10005000826089BF80E08FBD83E08EBD89B78068F4
:1000600089BF78948DED8CBD8BE08DBD00916400CF
:100070000A3009F013C080E080936400A7E68C91F9
:100080008F5F8C9300916700063009F007C080E015
:1000900080936700A5E68C918F5F8C93009165003B
:1000A0000A3009F007C080E080936500A8E68C91D3
:1000B0008F5F8C9300916800063009F007C080E0E4
:1000C00080936800A6E68C918F5F8C930091660008
:1000D0000A3009F007C080E080936600A9E68C91A1
:1000E0008F5F8C9300916900023081E009F080E01D
:1000F0008F9300916600043081E009F080E09F91C9
:100100008923882309F406C080E08093660080E09C
:100110008093690080990FC086E990E0F7D18099BB
:100120000AC0A5E68C918F5F8C9380E08093640079
:1001300080E08093670081990FC086E990E0E6D166
:1001400081990AC0A6E68C918F5F8C9380E08093A2
:10015000640080E080936700A0E30C9100FB81E0E5
:100160000EF480E08F93A0E30C9101FB81E00EF48C
:1001700080E09F918923882309F40CC080E080935C
:10018000650080E08093680080E08093660080E0F6
:10019000809369006BCFF894FFCF0F921F922F923C
:1001A0003F924F925F927F928F929F92AF92BF92B7
:1001B0000F931F932F933F934F935F936F937F936F
:1001C0008F939F93AF93BF93CF93DF93EF93FF935F
:1001D0008FB78F9300916000043009F003C080E076
:1001E00080936000A0E68C918F5F8C938FEF88BB2B
:1001F00000916000013009F009C0929A9398949898
:10020000959880916900809361002AC0023009F0BE
:1002100010C09298939A94989598A3E68C9187FB36
:10022000A8E38C9187F98C9380916600809361009C
:1002300017C0033009F009C092989398949A959842
:1002400080916800809361000BC0043009F008C001
:10025000929893989498959A809165008093610004
:1002600000916100013009F007C0EEEEF4E081E09A
:1002700090E0A2E665D182C0023009F007C0EEEE40
:10028000F4E082E090E0A2E65BD178C0033009F0B0
:1002900007C0EEEEF4E083E090E0A2E651D16EC03C
:1002A000043009F007C0EEEEF4E084E090E0A2E64E
:1002B00047D164C0053009F007C0EEEEF4E085E0F8
:1002C00090E0A2E63DD15AC0063009F007C0EEEE3C
:1002D000F4E086E090E0A2E633D150C0073009F0A8
:1002E00007C0EEEEF4E087E090E0A2E629D146C038
:1002F000083009F007C0EEEEF4E088E090E0A2E6F6
:100300001FD13CC0093009F007C0EEEEF4E089E0EF
:1003100090E0A2E615D132C000916100003081E08A
:1003200009F080E08F9300916000013081E009F0D6
:1003300080E09F918923882309F407C0EEEEF4E062
:100340008AE090E0A2E6FCD019C000916100003084
:1003500081E009F080E08F9300916000013080E03F
:1003600010F009F081E09F918923882309F406C0E9
:10037000EEEEF4E080E090E0A2E6E2D0A2E68C911E
:1003800080FB882780F9809580FBA8E38C9180F919
:100390008C93A2E68C9181FB882780F9809580FB65
:1003A000A8E38C9181F98C93A2E68C9182FB88273B
:1003B00080F9809580FBA8E38C9182F98C93A2E66A
:1003C0008C9183FB882780F9809580FBA8E38C9132
:1003D00083F98C93A2E68C9184FB882780F9809521
:1003E00080FBA8E38C9184F98C93A2E68C9185FB29
:1003F000882780F9809580FBA8E38C9185F98C9300
:10040000A2E68C9186FB882780F9809580FBA8E383
:100410008C9186F98C938F918FBFFF91EF91DF9133
:10042000CF91BF91AF919F918F917F916F915F918C
:100430004F913F912F911F910F91BF90AF909F903F
:100440008F907F905F904F903F902F901F900F90D4
:1004500018950F921F922F923F924F925F927F9228
:100460008F929F92AF92BF920F931F932F933F93C0
:100470004F935F936F937F938F939F93AF93BF93AC
:10048000CF93DF93EF93FF938FB78F938DED8CBD59
:100490008BE08DBDA4E68C918F5F8C93A3E68C914D
:1004A00087FB882780F9809580FBA3E68C9187F9EC
:1004B0008C938F918FBFFF91EF91DF91CF91BF917F
:1004C000AF919F918F917F916F915F914F913F91EC
:1004D0002F911F910F91BF90AF909F908F907F9021
:1004E0005F904F903F902F901F900F9018953F0670
:1004F0005B4F666D7D077F6F00003197F1F70895C0
:10050000689462F80895E89462F80895EF93FF9371
:10051000EE27E82BE92B31F0E8EEF3E03197F1F725
:100520000197D1F7FF91EF91089581E003C082E038
:1005300001C084E0C8950D9231968A95D9F7089547
:06054000E80FF91FF2CFE5
:00000001FF
